:020000040007F3
:108000009854002069840700718407007384070076
:10801000758407007784070079840700000000005A
:108020000000000000000000000000005584070070
:108030007D840700000000007F8407008184070022
:108040004198070083840700838407008384070026
:1080500083840700838407008384070083840700E8
:1080600083840700838407008384070083840700D8
:1080700083840700838407008384070083840700C8
:10808000838407009998070083840700838407008E
:10809000BD98070083840700C19807008384070008
:1080A0008384070083840700838407008384070098
:1080B00083840700838407000000000000000000A4
:1080C0008384070083840700838407008384070078
:1080D0008384070083840700838407000000000076
:1080E0000000000000000000000000000000000090
:1080F0000000000000000000000000000000000080
:10810000000000000000000000000000000000006F
:10811000000000000000000000000000000000005F
:10812000000000000000000000000000000000004F
:10813000000000000000000000000000000000003F
:10814000000000000000000000000000000000002F
:10815000000000000000000000000000000000001F
:10816000000000000000000000000000000000000F
:1081700000000000000000000000000000000000FF
:1081800000000000000000000000000000000000EF
:1081900000000000000000000000000000000000DF
:1081A00000000000000000000000000000000000CF
:1081B00000000000000000000000000000000000BF
:1081C00000000000000000000000000000000000AF
:1081D000000000000000000000000000000000009F
:1081E000000000000000000000000000000000008F
:1081F000000000000000000000000000000000007F
:10820000DFF80CD000F082F90048004765AC0700A9
:1082100098540020056885F308884068FF2464B2FC
:10822000EFF30585002D07D1EFF31481022291436E
:1082300081F31488A64600472546064621273FBA03
:10824000F0B40024002500260027F0B4F92040B245
:108250000047000030B450E8012F93B2C489234492
:108260008489A34228BF1B1B0489A34202BFBFF31A
:108270002F8F002007E0C3EA020340E80134002CFE
:10828000E9D14FF001000A6030BC704750E8012F7F
:10829000C2EA024240E801210029F7D1704730B418
:1082A00050E8022F1FFAA2F3C488A34202BFBFF313
:1082B0002F8F00200DE0C48923448489A34228BF66
:1082C0001B1BC2EA034340E80234002CE8D14FF004
:1082D00001000A6030BC704750E8022FC2EA224217
:1082E00040E802210029F7D17047034653E8022FE6
:1082F000D988B2EB324F4FF0000017BF92B241EA7B
:10830000014142EA014104E05A68B2EB324F08BF32
:10831000012043E80212002AE8D1704730B4044635
:1083200054E8000F0D4644E80053002BF8D11560C7
:1083300030BC704730B4044654E8000F40EA0105F1
:1083400044E80053002BF7D1156030BC704730B4BF
:10835000044654E8000F00EA010544E80053002BEE
:10836000F7D1156030BC704730B4044654E8000FB4
:1083700080EA010544E80053002BF7D1156030BCBA
:10838000704730B4044654E8000F00EB010544E8A0
:108390000053002BF7D1156030BC704730B4044651
:1083A00054E8000FA0EB010544E80053002BF7D17F
:1083B000156030BC7047000030B4044654E8000F2C
:1083C0000D4644E80053002BF8D1156030BC7047CF
:1083D00030B4044654E8000F40EA010544E8005375
:1083E000002BF7D1156030BC704730B4044654E818
:1083F000000F00EA010544E80053002BF7D1156097
:1084000030BC704730B4044654E8000F80EA0105E0
:1084100044E80053002BF7D1156030BC704730B4EE
:10842000044654E8000F00EB010544E80053002B1C
:10843000F7D1156030BC704730B4044654E8000FE3
:10844000A0EB010544E80053002BF7D1156030BCC8
:10845000704700001EF0040F0CBFEFF30880EFF32D
:10846000098003F083BF00000648804706480047A4
:10847000FEE7FEE7FEE7FEE7FEE7FEE7FEE7FEE7D4
:10848000FEE7FEE7E198070001820700202A04DBEF
:10849000203A00FA02F1002070479140C2F1200317
:1084A00020FA03F319439040704740EA01039B0709
:1084B00003D009E008C9121F08C0042AFAD203E059
:1084C00011F8013B00F8013B521EF9D27047D2B2BD
:1084D00001E000F8012B491EFBD270470022F6E7AD
:1084E00010B513460A4604461946FFF7F0FF20462A
:1084F00010BD30B504460020034600E05B1C9342EB
:1085000003D2E05CCD5C401BF8D030BD064C074D7B
:1085100006E0E06840F0010394E807009847103453
:10852000AC42F6D3FFF770FEA4DD0700C4DD070000
:108530002DE9F0438BB08046129D15F9046B00962F
:1085400014461F4689462B4602A81146424600F0B3
:10855000B8FC02A80146129A00F0A3FC404641462E
:1085600002AA129B00F08DFC2046214602AA129B13
:1085700000F087FC2B46384639464A46009600F004
:10858000A0FC02A83946129A00F08BFC02A8014612
:1085900042462B46009600F094FC02A80146224673
:1085A0002B46009600F08DFC2046214642462B4685
:1085B000009600F086FC484649462246129B00F091
:1085C00060FC2046414602AA2B46009600F079FC4A
:1085D000384639462246129B00F053FC384639464D
:1085E0004A462B46009600F06CFC204602A9324613
:1085F00000F031FE0BB0BDE8F083F0B589B01C4649
:1086000007460E461546684611461A4600F049FCD4
:10861000384639466A46234600F033FC68466946C8
:108620002A46234600F02DFC304631466A46234652
:1086300000F027FC09B0F0BD1AB1013A8B5C8354FD
:10864000FAE770472DE9F0478846B3F902101F4654
:108650000825CB1D202493FBF5F51F31954291FB96
:10866000F4F44FFA84F928BF15460646494600F04F
:1086700073FA2A4630464146FFF7DEFFB7F902306B
:10868000ED009D4220D9ED1A06EB840100228E42B6
:108690000AD251F8040D20FA05F313430B60C5F11B
:1086A000200300FA03F2F2E72437384631464A46FF
:1086B00000F05EFA012807D0304631463A464B4674
:1086C000BDE8F04700F01CBFBDE8F0872DE9F0479A
:1086D00093F9006092B0044689461046314615462B
:1086E000984600F06FFA002840F0978002A84946AB
:1086F000424600F0D6FB43460AA8214602AA00F0F3
:10870000C0FB02A80146424600F0CBFB4346484668
:1087100049462A4600F0B5FB08F1040728462946D9
:10872000424600F0BEFB204621462A463B460096C4
:1087300000F0F6FA284629462A463B46009600F005
:10874000EFFA284621462A463B46009600F0B9FB40
:10875000204621462A46434600F093FB2846214600
:1087600022463B46009600F0DBFA20463B46009648
:1087700021462A4600F0D4FA2368DB07204613D5A9
:10878000334621463A4600F0BBF931468246204640
:1087900000F054FD06F18043013B54F8230040EA09
:1087A000CA7044F8230002E0314600F047FD284635
:1087B0002146424600F075FB284629460AAA3B4658
:1087C000009600F07EFB284629460AAA3B46009602
:1087D00000F077FB0AA801462A463B46009600F0C7
:1087E00070FB204621460AAA434600F04AFB02A835
:1087F00002463B462146009600F063FB2046294690
:10880000324600F028FD28464946324600F023FD56
:10881000484602A9324600F01EFD12B0BDE8F087BE
:1088200000487047F4DC07002DE9F04FEFB01E461A
:10883000789C059023780493B4F9023092461F3354
:10884000202293FBF2F3DBB206939DF9187094F9A2
:10885000012007F1FF3926AB002543F829506EAB04
:1088600003EB89034EA88B46314643F8805C43F8FE
:10887000605CFFF7E1FE94F9012056A8B118FFF7FC
:10888000DBFE9DF910604EA8314600F09BF9804652
:10889000002840F02F8156A8314600F093F9054694
:1088A000002840F0258104F1240840464EA93A46AC
:1088B00000F05EF9012840F01D81404656A93A4675
:1088C00000F056F90128089040F014813B461EA89C
:1088D00056A9424600F03DFA0DF1380C6046594663
:1088E000524623464CF82950CDF80CC0FFF7AAFE9B
:1088F000DDF80CC00097604661461EAA4346CDF8DD
:1089000024C00DF5BC7900F0AAFA4346009716A8DA
:108910004EA91EAA00F0A3FA48463246059900F077
:108920009AFCB300039309EB030B039A059B58468B
:108930009918324600F08FFC04F144031946324680
:1089400036A8079300F087FC04EB860132463EA868
:10895000443104F1040A00F07EFC494600961EA84A
:1089600036AA534600F0ADFA4A465B4636A83EA901
:108970000094FFF7DDFD1EA801463346524600F085
:10898000E8F91EAA484659462346FFF736FEDDF8A9
:1089900024C0079B0B936046059B0C933946CDF88A
:1089A00014C00A95CDF8349000F026FC39460546EF
:1089B00016A800F021FCA842B8BF284685B2DDF811
:1089C00014C06F1E3FB26046394600F0C9FD3946FB
:1089D00010F1000916A818BF4FF0010900F0C0FD02
:1089E000002814BF0223002343EA09090DF1280BD4
:1089F00032465BF8297026A8394600F02CFC039B10
:108A00003246F9182EA800F026FC31461EA800F0C8
:108A1000A3F8023D089B1E93AEB237B2002F44DB91
:108A200023461EAAD4F8A45026A82EA9A847394642
:108A30000EA800F095FD3946051C16A818BF0125A3
:108A400000F08EFD002814BF022300231D430AAB53
:108A500053F8257037B39DF9105036A839462A4689
:108A600000F0F9FB039B3EA8F9182A4600F0F3FB3F
:108A700036A83EA91EAA2346FFF7BFFD46A826A991
:108A800036AA5346009500F01CFA36A83EA926AA3D
:108A90002EAB0094FFF74CFD1EA8014646AA2346C4
:108AA00000F0EFF9013EB6B2B7E79DF910501EA8ED
:108AB000014652462B4600F04CF9234626A82EA923
:108AC0001EAAFFF79AFD9DF91840404626A92246A6
:108AD00000F04EF8012805D026A80146424623465C
:108AE00000F00EFD26A84EA92A4600F056F802E036
:108AF000404600E028466FB0BDE8F08F000000005F
:108B0000C3F10803DB0070B501330446002003A560
:108B10005B1920C940CAAD1920C4184720C940CAF2
:108B2000754120C420C940CA754120C420C940CA2B
:108B3000754120C420C940CA754120C420C940CA1B
:108B4000754120C420C940CA754120C420C940CA0B
:108B5000754120C4404170BD10B5002253B28B4214
:108B600005DA1BB2002440F823400132F6E710BDBD
:108B700010B5013AD2B253B2002B09DB1BB250F848
:108B8000234051F823309C4204D8F2D2FF2002E067
:108B9000002000E0012040B210BD013A30B5D2B251
:108BA000002453B2002B09DB1BB2013A51F82350C9
:108BB00050F823306B401C43D2B2F2E7B4FA84F091
:108BC000400930BD10B500231A465CB28C4204DA6D
:108BD00050F8244001332243F7E7B2FA82F040090B
:108BE00010BD00002DE9F043A3B09846019112ABEF
:108BF0004146074610469146009300F0FDFAC0EB4F
:108C0000881086B2454C33B21C40002CBEBF04F124
:108C1000FF3464F01F040134202593FBF5F5EDB219
:108C20006DB2A4B202A8294624B2FFF795FF28B27C
:108C300002AB002C03EB800010DD002213464345FD
:108C400010D259F8235005FA04F10A4340F82320C2
:108C5000C4F1200225FA02F20133F0E74946424608
:108C600000F0F9FA0FFA88F502AB4FEA4509012442
:108C700003EB8505330444D40022114653B24B451F
:108C800022DA0DF1880E0EEB840E0DF1880C18B26D
:108C90005EF888EC0CEB83035EF820E053F8803C30
:108CA000C3EB0E035B1A734502D08CBF0121002178
:108CB000C4F1010E0DF1880C0CEB8E0E01325EF842
:108CC00088EC4EF82030D9E7621A544202A8414697
:108CD000544100F0B3FA22AA08F1FF3302EB8303F8
:108CE00002EB8802284652F8801C53F8802C013E83
:108CF00042EAC172414643F8802CB6B200F09EFAB7
:108D0000B8E722AB03EB8404384654F8881C42468B
:108D100000F0A1FA23B0BDE8F08300BF1F0000807F
:108D200070B59DF910401D4623460646FFF7E8FE44
:108D300030B9284631462246FFF71AFF012807D0EE
:108D4000304631462A462346BDE8704000F0D8BB85
:108D500070BDF0B50646A1B00F4608461946154647
:108D60001C46FFF72FFF20B130462146FFF7F4FEE7
:108D700073E068463946224600F06DFA08A8294695
:108D8000224600F068FA10A82146FFF7E5FE01230D
:108D900018A821461093FFF7DFFE684608A922466F
:108DA000FFF7E6FE002853D0009BDA0704D468469C
:108DB000214600F043FA26E0089BDB0704D408A80C
:108DC000214600F03BFA3DE000281EDD08AA2346BC
:108DD0006946684600F094FB6846214600F02EFA8A
:108DE00010A818A92246FFF7C3FE002805DA10A82C
:108DF00001462A462346FFF783FE10A8014618AA1B
:108E0000234600F07DFB10A81DE008A86A46234613
:108E1000014600F075FB08A8214600F00FFA18A8DB
:108E200010A92246FFF7A4FE002805DA18A801467B
:108E30002A462346FFF764FE18A8014610AA2346D7
:108E400000F05EFB18A82946224600F06BFCA4E760
:108E5000304610A9224600F0FEF921B0F0BD70B5F1
:108E600090B006469DF950401D466846234600F0E6
:108E70003AF8304669462A462346FFF7B3FE10B05B
:108E800070BD30B51C4691B0054693F90030684678
:108E900000F029F8D4F8AC3028466946984711B05C
:108EA00030BD30B5144691B0054692F900206846B1
:108EB00000F0DEF9D4F8AC3028466946984711B086
:108EC00030BD70B59DF910401D462346064600F0A2
:108ED00017FB38B1304631462A462346BDE870407C
:108EE000FFF70EBE70BD2DE9F04F08B4F8CA04B408
:108EF00051F8042BA3FB028940F8048B4FF0000AC1
:108F0000E4FB629A4FF0000BE5FB62AB4FF0000C04
:108F1000E6FB62BC4FF0000EE7FB62CE51F8042B7B
:108F20004FF00008E3FB628940F8048BE4FB629A8F
:108F3000E5FB62ABE6FB62BCE7FB62CE51F8042BBB
:108F40004FF00008E3FB628940F8048BE4FB629A6F
:108F5000E5FB62ABE6FB62BCE7FB62CE51F8042B9B
:108F60004FF00008E3FB628940F8048BE4FB629A4F
:108F7000E5FB62ABE6FB62BCE7FB62CE51F8042B7B
:108F80004FF00008E3FB628940F8048BE4FB629A2F
:108F9000E5FB62ABE6FB62BCE7FB62CE40F8049BFC
:108FA00040F804AB40F804BB40F804CB40F804EBB5
:108FB0000CBC052B00F01E810C68A0F11400A1F17F
:108FC0001401A2F1140252F804EB4FF0000550F81E
:108FD000046BE4FB6E5652F804EB50F8047BE4FBA0
:108FE0006E6752F804EB50F8048BE4FB6E7852F88D
:108FF00004EB50F8049BE4FB6E8952F804EB50F844
:1090000004ABE4FB6E9AA0F1140052F8044B51F843
:1090100004EB4FF0000CE4FB6EC540F804CB51F8B4
:1090200004EBE4FB6E5640F8045B51F804EBE4FB00
:109030006E6740F8046B51F804EBE4FB6E7840F87F
:10904000047B51F804EBE4FB6E8940F8048B51F883
:1090500004EBE4FB6E9AA0E80006062B00F0CA8041
:109060000C68A0F11800A1F11801A2F1180252F841
:1090700004EB4FF0000550F8046BE4FB6E5652F819
:1090800004EB50F8047BE4FB6E6752F804EB50F8F5
:10909000048BE4FB6E7852F804EB50F8049BE4FB7D
:1090A0006E8952F804EB50F804ABE4FB6E9A52F868
:1090B00004EB50F804BBE4FB6EABA0F1180052F8CF
:1090C000044B51F804EB4FF0000CE4FB6EC540F884
:1090D00004CB51F804EBE4FB6E5640F8045B51F806
:1090E00004EBE4FB6E6740F8046B51F804EBE4FB1F
:1090F0006E7840F8047B51F804EBE4FB6E8940F88D
:10910000048B51F804EBE4FB6E9A40F8049B51F891
:1091100004EBE4FB6EABA0E8000C072B6AD008B4AC
:109120000C68A0F11C00A1F11C01A2F11C0252F874
:1091300004EB4FF0000550F8046BE4FB6E5652F858
:1091400004EB50F8047BE4FB6E6752F804EB50F834
:10915000048BE4FB6E7852F804EB50F8049BE4FBBC
:109160006E8952F804EB50F804ABE4FB6E9A52F8A7
:1091700004EB50F804BBE4FB6EAB52F804EB50F880
:1091800004CBE4FB6EBCA0F11C0052F8044B51F878
:1091900004EB4FF00003E4FB6E3540F8043B51F85C
:1091A00004EBE4FB6E5640F8045B51F804EBE4FB7F
:1091B0006E6740F8046B51F804EBE4FB6E7840F8FE
:1091C000047B51F804EBE4FB6E8940F8048B51F802
:1091D00004EBE4FB6E9A40F8049B51F804EBE4FBCB
:1091E0006EAB40F804AB51F804EBE4FB6EBCA0E8B6
:1091F000001808BCBDE8F08F0139C9B24BB2002B92
:109200000BDA013111F0FF0315D059B201F180439F
:10921000013B50F82320002304E050F82330002BBA
:10922000EAD0EEE712B152080133FBE7481E03EB28
:10923000401080B200E0184600B2704700EB810198
:109240000023884206D251F8042D43EA52030B60F2
:10925000D307F6E7704730B5002463B2934206DACD
:109260001BB2013451F8235040F82350F5E730BDCC
:109270002DE9F04FB1E8005E06B4AAFB09124FF0E9
:109280000003EBFB69234FF00004ECFB69344FF063
:109290000005EEFB69454FF00006EBFB6A63ECFB53
:1092A0006A344918524176415B41A9FB09784FF075
:1092B000000949F1000918EB0108A0E88001AAFBA8
:1092C0000A78574158EB0608A0E88001EEFB6A4592
:1092D0004FF0000A4AF1000A4FF00001ECFB6B145A
:1092E000EEFB6B454FF00002EEFB6C255FEA59097F
:1092F0004941644152416D4149F10009EBFB6B3A30
:109300001AEB010AA0E80804ACFB0C6A66415AEBB0
:10931000020AA0E84004AEFB0E6A6E415AEB090A4D
:10932000A0E8400406BC052A00F0E680A0F1140085
:10933000A1F11401B1E8E043A5FB0E344FF00005A4
:10934000E6FB6E454FF00006E7FB6E564FF0000758
:10935000E8FB6E674FF00008E9FB6E784FF00009FC
:10936000DB1864416D4176417F4158EB080859F1A3
:10937000000950F804CB13EB0C0350F804CB54EB6A
:109380000C0450F804CB55EB0C0550F804CB56EB0D
:109390000C0650F804CB57EB0C0758F1000859F1B4
:1093A0000009A0F11400EEFB0E89A0E8F803062ADC
:1093B00000F0A280A0F11800A1F11801B1E8E04787
:1093C000A5FB0E344FF00005E6FB6E454FF000069E
:1093D000E7FB6E564FF00007E8FB6E674FF00008A2
:1093E000E9FB6E784FF00009EAFB6E894FF0000A46
:1093F000DB1864416D4176417F4158EB080859EB19
:1094000009095AF1000A50F804CB13EB0C0350F889
:1094100004CB54EB0C0450F804CB55EB0C0550F87E
:1094200004CB56EB0C0650F804CB57EB0C0750F866
:1094300004CB58EB0C0859F100095AF1000AA0F1CD
:109440001800EEFB0E9AA0E8F807072A54D0A0F106
:109450001C00A1F11C01B1E8E04FA5FB0E344FF058
:109460000005E6FB6E454FF00006E7FB6E564FF039
:109470000007E8FB6E674FF00008E9FB6E784FF0DD
:109480000009EAFB6E894FF0000AEBFB6E9A4FF081
:10949000000BDB1864416D4176417F4158EB0808B1
:1094A00059EB09095AEB0A0A5BF1000B50F804CB9F
:1094B00013EB0C0350F804CB54EB0C0450F804CB22
:1094C00055EB0C0550F804CB56EB0C0650F804CBCA
:1094D00057EB0C0750F804CB58EB0C0850F804CBB2
:1094E00059EB0C095AF1000A5BF1000BA0F11C00CA
:1094F000EEFB0EABA0E8F80FBDE8F08F0000000017
:10950000C3F10803DB0070B50133002403A500BFDD
:109510005B1920C940CAAD1B20C0184720C940CAEA
:10952000B54120C020C940CAB54120C020C940CAA9
:10953000B54120C020C940CAB54120C020C940CA99
:10954000B54120C020C940CAB54120C020C940CA89
:10955000B54120C06441B4FA84F0400970BD00BF39
:109560004A11012301F01F0150F822008B401840DE
:1095700070470000F0B50C4689B008220646FFF798
:109580006AFEE36A0393236B0493636B0593A36BF7
:109590000693E36B0793002769466A4608236846EB
:1095A000029701970097FFF7ABFA314605466A46E6
:1095B00008233046FFF7A4FA236B0393636B0493ED
:1095C000A36B0593E36B0693054469466A4608233B
:1095D00068460797FFF794FA314605446A46082320
:1095E0003046FFF78DFA236A0093636A0193A36AFA
:1095F0000293A36B0693E36B0793054431466A46D7
:1096000008233046059704970397FFF779FA636AB2
:109610000093A36A0193E36AA26B0293636B0393C3
:1096200004920693E26B236A059205440793314640
:109630006A4608233046FFF763FAE36A0093236B18
:109640000193636B0293236A0693A36A079305440D
:1096500031466A4608233046059704970397FFF77B
:109660004FFF236B0093636B0193A36B0293E36B38
:109670000393636A0693E36A07932D1A31466A4699
:109680000823304605970497FFF73AFF636B009372
:10969000A36B0193E36B0293236A0393636A0493BE
:1096A000A36A0593236B07932D1A31466A46082354
:1096B00030460697FFF724FFA36B0093E36B0193FB
:1096C000636A0393A36A0493E36A0593636B079346
:1096D0002D1A314630466A46082302970697FFF74F
:1096E0000FFF2D1A16D5304631460D4A0823FFF7D5
:1096F00007FA4519F7D410E0094831460822FFF768
:1097000037FA012809D030463146054A0823FFF7C9
:10971000F7FE2D1A002DEFD0F5E709B0F0BD00BF20
:10972000F8DC0700F8B5036813F0010506460F469C
:10973000144605D001463A462346FFF7E1F90546AF
:1097400030462146FFF77AFD45B104F18042013AE7
:1097500056F8223043F0004346F82230F8BD2DE998
:10976000F04115468AB00446884602A8002120220E
:10977000FEF7B6FE2E780323204641462A462F1DCB
:1097800076B20293FFF78DFB2046214602AA3B46A4
:109790000096FFF796FB2046214642462B46FFF7F0
:1097A00070FB00962046214605F184023B46FFF7F8
:1097B000B7FA0AB0BDE8F08100F01F020121914024
:1097C0004009800000F1E020C0F88012704700F0EE
:1097D0001F02012191404009800000F1E020C0F803
:1097E0000011704700F01F020121914040098000E4
:1097F00000F1E020C0F8001270474907090E002868
:1098000006DA00F00F0000F1E02080F8141D704728
:1098100000F1E02080F8001470470000BFF34F8F84
:1098200005480168054A01F4E06111430160BFF396
:109830004F8F00BFFDE700000CED00E00400FA05CB
:109840002DE9F0414FF48077384601F092FA012477
:10985000104EA50748B1384601F092FA0120C5F82C
:1098600008037470002000F015FD4FF4827738462D
:1098700001F07FFA00280BD0384601F081FA02206F
:10988000C5F80803B470BDE8F041012000F002BD46
:10989000BDE8F0814832002007480021C0F840119F
:1098A000C0F84411C0F84811C0F84C11C0F80011BC
:1098B000C0F8041103F046BF0010014003F090BE51
:1098C00010B50021054A084600F014FA002803D01C
:1098D000BDE8104000F00CBA10BD00009D9F0700CD
:1098E000F0B5AE480023021D01780125101D4FF090
:1098F000805406290BD11678360708D10678C6F3AE
:109900000316032E06D0042E04D0052E02D00629FD
:1099100007D00EE0B4F82463A14FC6F304263E60DE
:1099200002E01678360704D10678C6F30316032E34
:1099300002D0062904D00FE09B4F9A4E7E670EE0BE
:109940001678360708D10678C6F30316032E06D01C
:10995000042E04D0052E02D0062907D00EE0D4F83C
:109960004462924FC6F342363E6002E016783607F4
:1099700004D10678C6F30316032E02D0062906D0BA
:1099800011E08B4E376827F0807737600EE016784D
:10999000360708D10678C6F30316032E06D0042E28
:1099A00004D0052E02D006290AD011E04FF08046DF
:1099B000C6F80C31C6F810317C4E361F336002E019
:1099C0001678360704D10678C6F30316032E02D0A4
:1099D000062905D00CE0754F032664373E600AE087
:1099E0001678360704D10678C6F30316032E02D084
:1099F00006290DD014E06F4F05263E606D4E783677
:109A000035606C4E083633603F263F1D3E6002E0F5
:109A10001678360704D10678C6F30316052E02D051
:109A2000062957D062E0644E3668644F3E60624E4D
:109A3000361D36683F1D3E605F4E083636683F1D56
:109A40003E605D4E0C3636683F1D3E605A4E103605
:109A500036683F1D3E60584E143636683F1D3E60E6
:109A6000554E18363668554F20373E60524E1C36DC
:109A700036683F1D3E60504E203636683F1D3E60C2
:109A80004D4E243636683F1D3E604B4E28363668B4
:109A90003F1D3E60484E2C3636683F1D3E60464EA8
:109AA00030363668454F40373E60434E3436366870
:109AB0003F1D3E60404E383636683F1D3E603E4E8C
:109AC0003C3636683F1D3E603B4E403636683F1D93
:109AD0003E6002E01678360708D10678C6F3031612
:109AE000032E06D0042E04D0052E02D0062907D05E
:109AF00019E0D4F85812324A01F04F01116002E027
:109B0000117809070FD10078C0F30310032803D0A0
:109B1000042801D0052806D12A480168C90702D0C7
:109B20006FF00101016022487438016841F470014E
:109B30000160BFF34F8FBFF36F8F4FF01021D1F84B
:109B40000002002803DBD1F80402002822DA1E4AB2
:109B500015601E480468002CFCD01524C1F8004292
:109B60000568002DFCD0C1F8044201680029FCD032
:109B7000136001680029FCD0BFF34F8F0C48F03808
:109B80000168134A01F4E06111430160BFF34F8F94
:109B900000BFFDE710490F480860F0BDE00F00F07E
:109BA000403501400DF0ADBA00C007403C05004013
:109BB000FCED00E0105600400404001020C50040F9
:109BC000E40E00400004004004E5014000E40140D0
:109BD0000400FA050090D003B028002002E008C875
:109BE000121F08C1002AFAD170477047002001E017
:109BF00001C1121F002AFBD170470000012120285B
:109C000003DA81400548014003E0402802DA2038A9
:109C1000814009B10120704700207047FC06FFBD5C
:109C2000082806D228B1012803D0042801D0012039
:109C3000704700207047800701D000207047012046
:109C40007047C3688B4206D811440069491E81429F
:109C500001D80120704700207047000000B5224B5A
:109C60008DB00DF1240C0FCB8CE80F001621ADF850
:109C7000201002218DF80010012206208DF801200D
:109C80008DF8020003208DF803008DF80410592090
:109C90008DF80500FE208DF8060008A90DF10900D9
:109CA0007DDF68B9BDF82000411C8DF8071009213F
:109CB00009308DF80810C1B200231A46684672DFD9
:109CC00000280FD174DF012109A873DF002809D112
:109CD0004FF0A0404FF40031C0F80C15122002F0F4
:109CE00010FA00200DB000BD58DA0700FFF796FD0E
:109CF000FFF794FD2DE9F84F254C81469246608888
:109D00000E46814241D800274FF6FF788DF800704B
:109D1000684600F005F922786078A188884201DA67
:109D2000401C00E00020C0B2904204D19DF8000029
:109D300000F01AF927E065786078884201DA401C63
:109D400000E0002060709DF8000000F00DF945452E
:109D500019D0A068B9F1000F40F835A00DD066B158
:109D60006188E068324605FB01004946FEF79DFB2D
:109D7000A06800EBC500868002E000EBC50087808C
:109D80000020BDE8F88F0420FBE70920F9E7000078
:109D90007C28002010B50E4C03E0401C00E00020A1
:109DA000207020786178814210D022786188E06844
:109DB000A36802FB010003EBC20153F8322089883B
:109DC00090472078A1888842E9DAE6E710BD0000D4
:109DD0007C28002030B5CB0008339DB293074FF0AC
:109DE000000401D0072030BD044B9A602A44DA6099
:109DF0005C701C7058809980002030BD7C28002049
:109E0000074B9B7823B12AB120B10068037C1BB1BA
:109E10000820704707207047417442610020704756
:109E20005C32002070B503F03FF9104800240B218C
:109E3000047044700E4D817014206C602C706C7036
:109E4000FFF7BAFC07211420FFF7D7FC1420FFF717
:109E5000BEFC0848046007211120FFF7CEFC05482E
:109E6000001F0068A860002070BD00005C32002068
:109E70008C280020081501402DE9FC47DFF8789078
:109E800099F8023073B368B3052902D20720BDE800
:109E9000FC87436933B3437C012B25D0002704465C
:109EA0000025884616468DF80050684600F038F8C0
:109EB00001A803F0A3FCC8B1012101700F4944605F
:109EC0000968C0E90218C0E904769DF8040089F821
:109ED00001009DF8000000F047F81420FFF782FC15
:109EE0002846D4E70820D2E70F46D8E704259DF896
:109EF000000000F039F8F3E75C320020041501405F
:109F00000649897839B130B1416921B10021017424
:109F1000022103F0F3BB0820704700005C320020F0
:109F200030B5EFF3108172B60D4A9468012324B165
:109F30000370002900D162B630BD93604FF0E0237A
:109F4000D3F88051074C25401560C3F88041D3F801
:109F5000844154605A17C3F8842100220270E8E754
:109F600068330020FC06FFBD0B498A68002A11D027
:109F700000280FD1EFF3108072B60B684FF0E0228B
:109F8000C2F800314B68C2F8043100228A60002810
:109F900000D162B6704700006833002002F07AB941
:109FA00030B50546154C85B04FF6FF702080012076
:109FB0008DF812004FF65960ADF810002A4604A93A
:109FC0000120A0DF002817D10D4B0FCB8DE80F002B
:109FD000A91C684662DF00280ED1284600F0E8FB85
:109FE000002809D1284600F099FA002804D1A06879
:109FF00040F00100A060002005B030BD68280020BE
:10A0000068DA07000D4810B502880024A2F57F41E8
:10A01000FF390CD0816841F00401816013211046A2
:10A0200076DF040008D1064800F0DAFF03E074DFB1
:10A03000112002F066F8204610BD000068280020BC
:10A04000400D030010B5112002F053F8122002F069
:10A0500050F8112002F055F8122002F052F80120B9
:10A0600000F0CEF8002818D101F022FE38B10B48DC
:10A0700001F012FE0A48816841F00201816000F09F
:10A0800095FC002809D105482838FFF789FF0028EA
:10A0900003D1BDE81040FFF7E1BD10BD2C2D00201D
:10A0A00068280020FEB5514D0446008800212B8809
:10A0B00004F1080623287DD024DC13283BD014DCCF
:10A0C00001285FD0102827D011280DD1122002F0CE
:10A0D00018F8287A400704D4FFF7C0FD08B1FFF74D
:10A0E00007FE4FF6FF702880FEBD14285ED01A28A8
:10A0F00064D01F2836D02128F6D10091A088694667
:10A100008FDF2AE050380828EED2DFE800F05D3F0C
:10A11000570404642F10E7E74FF0A0414FF480206C
:10A12000C1F80C05112001F0ECFFA088DBE7BDE8C9
:10A13000FE4001F0F9BC2E486A4642F6052100684F
:10A14000009002A801901846A5DF08B1FFF7D0FDE6
:10A1500000231A46852128887FDF0028C4D0FFF716
:10A16000C7FDFEBD3146184675DF05E0A079002821
:10A17000F7D11321184676DF0028F2D0BDE8FE4063
:10A18000FFF7B6BD0021184666DFF5E7A079002885
:10A19000E7D02146174802F0B5F90028E1D003B016
:10A1A0003146BDE8F040134802F00EB900210A46DE
:10A1B000A08800E013E00B4686DFDDE70023A088DF
:10A1C0001A461946A9DFD7E703B02146BDE8F0409B
:10A1D000084802F0E1B9A0881721ADDFCCE7009173
:10A1E0000191A0880022694690DFB6E76828002028
:10A1F00050DA0700042D0020007800F001007047BD
:10A200007FB50024009401940294039418B101F0E6
:10A2100065FB00282CD1174813DF002828D102F055
:10A2200003F808B1FFF764FD684601F0ABFF0028B2
:10A230001ED1012501948DF804508DF8054002943B
:10A2400003948DF8064001A94020009A69DF01942B
:10A250008DF804501720ADF806000294039401A96C
:10A260002320009A69DF002802D1684601F094FF9C
:10A2700004B070BD0080070010B543689C184460AE
:10A2800021B905E013F8010B01F8010B521EF9D2B8
:10A29000012010BD70B5084C050009D010342168AC
:10A2A000002907D008682060496828468847F6E7F3
:10A2B0000834F4E770BD0000483200202DE9F05F5B
:10A2C00026484168F1B3DFF898B00E688146DBF8A4
:10A2D000004087688078E11B21F07F45ED1CB0B914
:10A2E000DFF880804FF48030C8F84403C8F80403D6
:10A2F0001120FFF761FA1120FFF769FA4FF0010A08
:10A30000C8F800A02F2000F0B1FE89F802A0B542E5
:10A3100000D23546124BE8193C3320F07F401860DC
:10A32000DBF800105A46091B21F07F41001B20F08A
:10A330007F40C91C81420FD9106818602F2000F09F
:10A3400095FE00E004E0BDE8F05F1120FFF74ABA97
:10A35000BDE8F05F02F0A8BEBDE8F09F8C280020A9
:10A360000415014000100140F0B54FF0FF3622B156
:10A370001268D24300230A4D0DE03246FAE7C45C6E
:10A3800062400824D70700D037462F4087EA5202A0
:10A39000641EF7D15B1C8B42F1D3D043F0BD0000AB
:10A3A0002083B8EDF0B5146906468DB020681546D7
:10A3B000271DE0B1022920D00A2000906B4609AA8F
:10A3C000304602F077FD00280FD009A901A8009AB5
:10A3D00002F062FC01AE96E80F0005AE86E80F00C1
:10A3E000236869683A4605A898470DB0F0BD0DB0DE
:10A3F0003046BDE8F04002F0C3BC6946304602F08A
:10A4000055FC0028F1D0236869683A4668469847A9
:10A410000028EAD002980028F5D101987060012048
:10A42000E3E753685B7813F0C00303D0402B03D0FD
:10A430000020704700F002B8FFF7B4BF2DE9FF41DC
:10A440000B465168064614464878334D00F00F021B
:10A4500010F0300055F8225006D0102806D02028E1
:10A4600008D0302856D13EE022694DE061690120D4
:10A47000087047E0022B28D1042A26D84FF00108A3
:10A4800069463046676902F011FC00281AD009E0DD
:10A490000B79226913FB00226846A84770B138780F
:10A4A000401C3870029820B1616838784A7990422F
:10A4B000EED301987060029860BB02E04FF0000894
:10A4C000F7E7404604B0BDE8F081D4E904300F79E5
:10A4D000027817FB023349798A421BD2521C027060
:10A4E0001A46616810E008786169072A087009D186
:10A4F000606801792069FDF7F1FF60682169806873
:10A5000002F0EFFB2269616804B03046AC46BDE85A
:10A51000F04160470020D5E7D0DC070010B58EB0D1
:10A5200004461C216846FDF7D9FF142108A8FDF751
:10A53000D5FF9DF80010002041F0180107908DF81C
:10A540000010A1788DF836100121ADF834109DF877
:10A550001C1004F10C0321F0FF018DF81C109DF874
:10A560001D1008AA21F00F01491C21F0F001103143
:10A570008DF81D109DF81E1021F00601891C41F078
:10A5800011018DF81E100DA9089107A90991172135
:10A59000ADF82C100C9020886946A2DF0EB010BDDB
:10A5A0001FB50E4800F15C01826B684602F074FB37
:10A5B0000B489DE80E0080E80E00094909480B4A47
:10A5C000C86009490020086048600949044802F051
:10A5D000FDF8002800D0012004B010BD703000202C
:10A5E000542C002001CB070040280020C828002060
:10A5F000E0D9070005490A6812B10A68521E0A60CC
:10A600000169002900D00847704700007428002025
:10A610002DE9F04799461600054600F104044FF075
:10A62000000110D0B9F1000F0DD094F88F0018B1CF
:10A6300094F89000012854D0207A20B1E0683428A2
:10A6400003D006203AE0042038E094F85520032A8D
:10A6500011D000204FF44057237C08E004EB800C1D
:10A66000B7F80C80DCF814C0C44504D0401C834209
:10A67000F4DC072022E04A487AB1012A07D0022AF6
:10A6800001D0032ADFD121780029DCD0C1684AB18A
:10A69000022A0CD0032A0DD109E021780029D2D05A
:10A6A0008168F4E76068884204D2052006E06068AB
:10A6B0008842FAD995F8A00020B10B20BDE8F047F8
:10A6C00000F06EB9374F384B4A463146386800F0D3
:10A6D000F3FB30B9344895F8A1200838416891421D
:10A6E00002D00A20BDE8F087006805F1A201FDF75D
:10A6F000DCFE2D4B2C4AD7F80200083BA2F11001DA
:10A7000000F090FB08B10520ECE7274D0020283D24
:10A71000E86094F85510C9B1012924D023480229D2
:10A72000C0F5FC2018D003298DD194F85C100029C5
:10A7300089D094F85610002985D0A26D216E531847
:10A74000EB6042B339B3814223D812E094F864003D
:10A7500000289AD0A06E0BE094F85C10002994D0E9
:10A76000216EE960EFE794F8560000288DD0A06DC7
:10A77000E8600D482022083004F16F010068FDF701
:10A7800094FEE86838B1084A0021203A00F07AFFC8
:10A7900018B10420A6E70320A4E70120A2E70000E7
:10A7A0007030002044DA070058280020008007009D
:10A7B00010B58EB004461C216846FDF78FFE1421AB
:10A7C00008A8FDF78BFE9DF80010002041F0040161
:10A7D00007908DF80010A1788DF836100221ADF8A1
:10A7E00034109DF81C1008AA21F0FF018DF81C10F0
:10A7F0009DF81D1021F00F01491C21F0F0011031CE
:10A800008DF81D109DF81E1021F00601891C41F0E5
:10A8100001018DF81E100DA9089107A909911421B5
:10A82000ADF82C100C902088231D6946A2DF0EB0D5
:10A8300010BD00000E4910B50A784C780023A242E2
:10A8400012D0521CD2B20A70022A00D10B70084AF0
:10A850000B780C3252F8232002608868104420F0F4
:10A860007F408860012010BD0360002010BD000003
:10A870008C2800202DE9F84380461F4615460E46D9
:10A8800000240D4800F050FA38B11120BDE8F883DB
:10A8900006EB043001F03CFC641CAC42F8D10648E5
:10A8A00000F03BFA2B46324602214046009700F06A
:10A8B0002BF80020EAE70000A02800202DE9F8434B
:10A8C000104D0F4680461E4691466946286800F0A6
:10A8D000F8F9040014D01C21FDF700FE01202071BE
:10A8E000C4F81490380BC4F80080C4E902606946CB
:10A8F000286800F007FA02F0BBFA0020BDE8F883F0
:10A900000420FBE7FCDA07002DE9F04186B004469D
:10A910008068DDF830801D4616460F4600280CD0B2
:10A9200014216846FDF7DAFDCDE902658DF8007067
:10A93000CDF81080A1686846884706B0BDE8F08170
:10A9400030B50446006885B00D46806800281CD0EC
:10A9500014216846FDF7C2FD0195A0680490207996
:10A9600010B101280DD104E001208DF8000020690C
:10A9700004E002208DF80000E068000302906069A6
:10A980000390206881686846884705B030BD0000A4
:10A990000249002208780A707047000078280020D9
:10A9A000014908700B2070477828002010B586B048
:10A9B00000249DF80000019420F00F00401C20F0BE
:10A9C000F00010308DF80000029403A86DDF00281D
:10A9D00025D19DF80D00401C8DF80D0003A86CDFFB
:10A9E00000281CD10F48007A800703D50E48011DAE
:10A9F000806901E00DA1072082B268467CDF002853
:10AA00000DD10620ADF804001820ADF80600ADF811
:10AA100008404FF4C870ADF80A0001A87ADF06B00C
:10AA200010BD0000682800202C2D002044667554BD
:10AA30006172670010B501F03FFC08B140DF10BD46
:10AA4000054901200860012000F0A2F90028FAD190
:10AA50000249487010BD0000040000404832002048
:10AA600010B50A4C2068FFF74BFA08B1FFF740F920
:10AA700000224FF470112068FFF7FEF9002803D080
:10AA8000BDE81040FFF734B910BD000078DA0700C8
:10AA90000149416000207047D0DA070038B504460C
:10AAA0000A4801216A46FDF793FC68B908486060CE
:10AAB00001F002FC05491C23FC2208740448FC39FF
:10AAC000001F006800F0EAF8002038BD7034002054
:10AAD00000DB070002480068002800D00120704712
:10AAE000A02800200248007A002800D001207047EA
:10AAF00070340020800701D000207047012070478B
:10AB00000268134602E08A4204D01268002AFAD191
:10AB10000B600160704770B5054608680C464A68CE
:10AB200086682846314601F0FDFF6068286104F11F
:10AB30000C00686170780221B1EB901F01D1241DD7
:10AB40002C6170BD06490120086006480168C1F308
:10AB500000410029FAD104490020887070470000A4
:10AB60000C00004018040040483200202DE9F04756
:10AB7000394E002780463D46DFF8E090D6F804A025
:10AB800057E003D00446D0F81C8035E099F8002047
:10AB900002EB4201521CD2B289F8002009EBC1013C
:10ABA00099F80230091D9A4201D189F8005048688D
:10ABB0000A780446012A12D0022A02D0032A3BD185
:10ABC00008E002F06BFD00B10127257434E0057444
:10ABD000C06900E070680028F9D170602CE0207C2A
:10ABE00050BB88686060C868A0600869E060486918
:10ABF000A061F07800B165606268B168184B501AC6
:10AC000020F07F40984202D2A168084406E0881AEA
:10AC1000A16820F07F40814202D9081A206000E03C
:10AC2000256065600120A56020742046E56102F082
:10AC300017FDB8F10000A4D199F8001099F80100AF
:10AC40008142A3D117B97168514502D00120BDE8F6
:10AC5000F0870020FBE700008C2800205C320020F9
:10AC6000FFFF7F0010B500F07CF808B1FEF7D6FDBD
:10AC70004FF44050806800F05DF8002010BD4FF0A8
:10AC8000A0414FF08070C1F80805704710B5FDF77E
:10AC90002CFB08B1002010BD112010BD10B531B142
:10ACA000B2FBF3F403FB14241CB1092010BD0E20E9
:10ACB00010BD01600021416081608281C38108462E
:10ACC00010BD70B50C460546FDF7C4FA002802D049
:10ACD00021882868084470BD10B50A8849888A42CE
:10ACE00003D1FDF7F9FA012010BD002010BD70B5A9
:10ACF0000C460546FDF7D3FA002802D06188286883
:10AD0000084470BD10B50A8849888A4203D1FDF70E
:10AD1000BDFA012010BD002010BD08B500216A4613
:10AD2000FDF715FB009808BD08B501216A46FDF73F
:10AD300001FB08BD10B5044600F0D0FD00280FD17E
:10AD40004FF0E021401EC1F88001C1F8800220468A
:10AD500013DF002804D12046BDE81040FDF75ABAA1
:10AD600010BD10B500F080FD002801D100F0F2FC0C
:10AD700010BD00F180400068002800D0012070471D
:10AD800008B500F18040002101600068009008BD16
:10AD90000549096840F4803001F00111814201D178
:10ADA00001207047002070470C0400402DE9F0039B
:10ADB00000F0FF0C0023182530221C263824202701
:10ADC0004FF04009BCF10A0F25D2DFE80CF0240552
:10ADD0001D0B2015181D0B2014224A60282211E09B
:10ADE0008A6002E0C1E900468C60BDE8F003C0F370
:10ADF00007200C3100F0D1B84A60602202E0422204
:10AE00004A6084220A60EBE7C1E90025E8E7C1E96E
:10AE100000974A46E4E74B600B608B60BDE8F003A7
:10AE2000062070472DE9F04186B01C4615460E46B7
:10AE30008046FDF7F5FC074646B33DB334B33068B2
:10AE400030B3296821B3216811B3FFF753FEF8B17D
:10AE50002868FFF74FFED8B12068FFF74BFEB8B166
:10AE600001A94046FFF7A2FF00280CD170680199A4
:10AE7000884207D16A680498824203D160680399C6
:10AE8000884207D0092006B0BDE8F0810E20FAE71D
:10AE90001020F8E708F0FF00042801D00620F2E7B0
:10AEA0000097236829683068FDF7BEFC08B10020D0
:10AEB000E9E70B20E7E70000F0B506461A48A1B025
:10AEC0001C004068029004A817460D46019008D067
:10AED0003DB1206838B1F0B2052806D0062021B077
:10AEE000F0BD0E20FBE71020F9E7694600F055F8A9
:10AEF0000028F4D160680099884201D00920EEE76B
:10AF000001A9304600F035F80028E8D13A46294634
:10AF100001A800F059F80028E1D1224601A93046E5
:10AF200000F004F8DBE70000C8DA0700F8B51446C3
:10AF3000054621B11CB1486870280DD101E00720F9
:10AF4000F8BD0E68E8B2694600F027F80028F7D18E
:10AF500060680099884201D00920F8BDC5F3072038
:10AF600028B100223046216802F060F9F8BD0122C4
:10AF7000F8E731B10A6832B14968702905D2092071
:10AF800070470E20704710207047C0B2052801D0CE
:10AF900006207047104602F0D1B91422082811D2B9
:10AFA000DFE800F01004100406080C0E0A6003E04D
:10AFB0001C2000E020200860002070473020FAE7C5
:10AFC0004020F8E70620704728B121B14368702B74
:10AFD00003D20920704707207047006802F06EBA5C
:10AFE00000283ED01F49204A096800BF00BF00BFAB
:10AFF00000BF00BF00BF00BF00BF91422FD000BF05
:10B0000000BF00BF00BF00BF00BF00BF00BF00BF48
:10B0100000BF00BF00BF00BF00BF00BF00BF00BF38
:10B0200000BF00BF00BF00BF00BF00BF00BF00BF28
:10B0300000BF00BF00BF00BF00BF00BF00BF00BF18
:10B0400000BF00BF00BF00BF00BF00BF00BF00BF08
:10B0500000BF00BF00BF00BF00BF00BF00BF01387E
:10B06000C3D17047B02800200024F40000283ED04F
:10B070001F49204A096800BF00BF00BF00BF00BFD2
:10B0800000BF00BF00BF91422FD000BF00BF00BF74
:10B0900000BF00BF00BF00BF00BF00BF00BF00BFB8
:10B0A00000BF00BF00BF00BF00BF00BF00BF00BFA8
:10B0B00000BF00BF00BF00BF00BF00BF00BF00BF98
:10B0C00000BF00BF00BF00BF00BF00BF00BF00BF88
:10B0D00000BF00BF00BF00BF00BF00BF00BF00BF78
:10B0E00000BF00BF00BF00BF00BF0138C3D1704721
:10B0F000B02800200024F4002DE9F05F244C4FF428
:10B1000040594FF48058216B666AD9F80830771A95
:10B1100003EB010B01EB000A4546AF4200D83D4668
:10B1200000220121584600F0E5FA00282ED1002324
:10B130002A465146584600F0FBFA002826D12A46F6
:10B140005146584600F09EFB00281FD1206B284432
:10B150002063002000F00AFEAB44AA447F1BDBD131
:10B1600000223146D9F80800FFF7FEF8A16A8142B3
:10B1700003D10121A661C4E907010548243000F08C
:10B1800075FBBDE8F05F002000F0F0BDBDE8F09F6A
:10B190007030002010B50A4C206A01280BD1E069FC
:10B1A00058B14FF44050A16980680022FFF7DCF8E5
:10B1B000E169814201D0002010BD012010BD0000D6
:10B1C0007030002070B506460C4608681049496B7F
:10B1D000451AA068AC2806D12A46A6F580410D483C
:10B1E00000F050FB58B12A4631460A4800F04AFBAD
:10B1F00028B129463046BDE8704000F051BB2046DA
:10B2000000F034FBBDE87040034800F0AFBD000023
:10B21000703000200080070051CF070000207047E9
:10B220002DE9F041454C0B780F4616460125D4E92F
:10B230000E102A02DFF80881072B7DD2DFE803F029
:10B240007C04213C1D7C7700B86820B1904204D971
:10B250000420BDE8F0810320FBE73A480068FEF7D0
:10B260004FFE3648002688F8036020213830FDF76D
:10B2700035F92663B868A06355E07060206CB06053
:10B2800053E0BA6813188B4203D97060206CB06029
:10B29000E1E72A4B79685C331844FDF706F9E06B67
:10B2A000B968264A0844E063D7E901014032FFF754
:10B2B0005BF82064E06BE0E7884201D00820C8E733
:10B2C00098F80300444608B10120C2E7FFF768F987
:10B2D000012824D11C4890F8A410B1B100F5637185
:10B2E00090F8AA20A830012A01D005200BE0144ACA
:10B2F00010320CCAFFF78CF9012804D1002000F0AD
:10B3000035FD70B10A2005460DE0007838B1032004
:10B31000FFF746FB0546012803D004E00CE00520BA
:10B3200097E70120E070FFF79BFB284691E77060EC
:10B33000206C3260B060F8E70225F6E7703000203C
:10B3400030280020C4DA0700C828002030B40B4B96
:10B3500002464FF440501C69816803F11800012C2B
:10B3600008D05C6934B19B690C3003F6FF736FF34E
:10B370000B03194430BC00F003B80000703000200B
:10B380002DE9F04116460C4682680021DFF87C80EA
:10B390000546012A09D040460127806CA52A0CD019
:10B3A000AA2A1BD0AC2A1ED120E0D8F8140001280C
:10B3B00019D12046FFF7A0FE14E000B1044629464B
:10B3C000204600F0CDFB010006D1284600F04EFAE1
:10B3D0000F4800F0CBFC16E0376004E02946204619
:10B3E000FFF7F0FE01460846BDE8F08100B10446D3
:10B3F0002946204600F0B4FB28B9D8F83400294685
:10B400002044FFF7DFFE0146E6E700007030002031
:10B4100051CF07002DE9F05F894E91F800C0874FAA
:10B420000C461546D6E91410FA78B36C4FF0010BB0
:10B430004FF4805A4FF00009BCF1070F7ED2DFE8CD
:10B440000CF0FA0433D7D3FAF500A168B1B37B4B03
:10B450000D05DB6802D045189D4237D151452BD8E8
:10B46000002A6CD00144994269D8F16CB164A1689A
:10B47000306571643063716909B9C6F82090B97894
:10B48000491C01F00301B970A7F80690A168BA68D9
:10B4900001F6FF711044090B002200F02BF900287F
:10B4A0007ED00520BDE8F09F6960B06CA860002ADE
:10B4B00045D0A168802902D90420F3E706E0306D69
:10B4C000726D0844801A726C904201D90320E9E73A
:10B4D0005B4A60684832FEF747FFB064306DA2688F
:10B4E000B046104430656860B06CA860F888A26807
:10B4F000DFF850A111183E46802905D2B77861685F
:10B500000AEBC713184436E0C0F18001B3788FB25C
:10B510000AEBC31210443A466168FCF7C6FFF08894
:10B52000384482B2F280A068C01BA06060683844D2
:10B5300060604746D8F83000B16801E07BE05BE02E
:10B54000B37808440AEBC311002300F0F1F840B3CC
:10B55000F86CB864786D38656860F86CA860B0788D
:10B56000401C00F00300B070A6F80690A26882B3F9
:10B570000AEBC0106168FCF798FF2089F188084445
:10B580000204F080120C4ED0D8F85410D8F83000D5
:10B59000D8F84430411A11444446994243D301E05B
:10B5A0003FE017E0B168B37808440AEBC311002309
:10B5B00000F0BEF898B1E06CA064606D2065686032
:10B5C000E06CA860B078401C00F00300B070A6F8F2
:10B5D000069028E0F188386B08443863BFE7F188AB
:10B5E000206B08442063EDE76960B06CA8601AE046
:10B5F000726C081A904201D0082053E7C6F84490B4
:10B60000F3640020716500F0B1FB08B10A2049E73E
:10B61000306DF968884204D10A48E03800F06AF9D0
:10B620008346FFF71DFA58463CE7FFE7AB60306DF5
:10B63000C5E900A0F7E74FF0020BF4E7302800203F
:10B6400070300020542A002010B5FFF7E7FD90B9B4
:10B650000A480068C0B2B1280DD00948816D01299F
:10B6600001D0002010BD00218165084600F07EFB5E
:10B6700008B1FEF73DFB012010BD00001C05004095
:10B6800070300020F0B54FF010235C694FF4405348
:10B690009B68E61AA6F5405682B186421BD3144C2D
:10B6A0001360A4F1180300251F6A012F08D01D6143
:10B6B0005D616560A56020600020F0BD0720F0BDE1
:10B6C000276807F6FF776FF30B07A6EB070C012639
:10B6D000604505D909B10420F0BDC3E90465E8E778
:10B6E000C3E904561168024C39440C341160E0E798
:10B6F00088300020054B30B41C68641C1C60134665
:10B700000A46014630BC024800F024BC74280020E0
:10B71000B428002008B1034900E00349002203488F
:10B7200000F03FBC0CDB0700DCDA0700B428002087
:10B7300038B5064C25686D1C2560009313460A46F3
:10B740000146034800F0A2FC38BD00007428002028
:10B75000B428002038B50020009000F0DDFA00F099
:10B7600055FB08B1FEF7C4FA002000F089FB36480B
:10B770000168C1F300410029FAD0344A03204FF098
:10B78000A041C2F8000701242006C1F80805FEF711
:10B7900049FB08B1FEF7ACFA2D4A00212D48FEF70F
:10B7A0002FFB08B1FEF7A4FA2A482B4A0121001DFD
:10B7B000FEF726FB08B1FEF79BFA2648274A002130
:10B7C0000830FEF71DFB08B1FEF792FA6846FFF756
:10B7D000BDFD00B10094FFF737FF00B10094204990
:10B7E00000200860009890B9FFF7D4FC78B100F011
:10B7F00039FA00280AD1FFF7CDFC30B100F074FB14
:10B800004FF440508068FFF795FA002038BD154A84
:10B8100010210820FEF7DEFA08B1FEF769FA0D489C
:10B8200000224FF470110068FEF726FB0028EDD1CE
:10B8300000F0D6FA0028E9D100F02CF901F0B2FEB0
:10B84000FEF7A8FA3EDFFBE7180400406000005056
:10B850003DBB070078DA0700D9D107007FAC0700AD
:10B860001C050040A82D0020002070470021016029
:10B870004160816002480163416301614161704739
:10B88000703000201FB5054B01AC92081B6A009375
:10B8900084E80700684618DF04B010BD84DA0700AA
:10B8A0001FB58908002201AB009283E807006846B3
:10B8B00018DF04B010BD00001FB59208930502D038
:10B8C000092004B010BD044B1B6800930392CDE91E
:10B8D0000110684618DFF4E784DA07001FB5044B4F
:10B8E0000FCB8DE80F00684618DF04B010BD0000D4
:10B8F00094DA07002DE9F047064690F86D0001271D
:10B90000DFF87C81032801D0092013E05D485C4BFF
:10B91000D8E9021200683033FFF7CEFA00B10A27E7
:10B9200057482022303006F16F010068FCF7E1FD36
:10B9300018B10C20FFF734F80746534D6A6922B15D
:10B94000012A05D00A20BDE8F0874F4C183401E0E9
:10B950004D4C243496F855304FF0010A4FF0000951
:10B96000ABB34A494FF44050012B05D0022B38D0DD
:10B97000032B19D00A2736E00278142A01D940692E
:10B9800000E00020D8F80820B0FBF1F002F50052EA
:10B990001378142B01D9526900E00022B2FBF1F1B7
:10B9A00088421ED005271EE00378142B01D9406978
:10B9B00000E00020D8F80830B0FBF1F003F50053A8
:10B9C00093F800C0BCF1140F02D95B6901E008E0F4
:10B9D0000023B3FBF1F1884203D0012A01D1C5F85D
:10B9E0002090012F05D0C4F808904846C4F8049070
:10B9F0002FE096F8550088B1012817D0022817D0FB
:10BA0000032818D00420FEF7CBFF074696F8550010
:10BA1000B0B1022817D0032817D114E0C4F808A049
:10BA200068690128F2D1C5F82090EFE7A52003E06E
:10BA3000AA20A060EAE7AC20A060B06D6863E5E7EB
:10BA40007068A86001E07068E860A86C6060D8F871
:10BA50000C0020600C4820213830FCF73FFD0A48DC
:10BA6000FF22FC215C30FCF732FDC5F8309088F8ED
:10BA700005A0074800F07AF900B10A27384662E7C6
:10BA80003028002044DA07007030002040420F00C8
:10BA9000C1C4070070B50120FFF73CFE00281DD18E
:10BAA0000F4CA06B78B1FEF77BFD60B10D4D206AA5
:10BAB00068B9A06958B10B4A00210832E860FFF765
:10BAC000E1FD0120E8700020FEF76AFF05E0E06A72
:10BAD00018B9A06908B1606AEDE7002070BD0000E8
:10BAE000703000203028002030B40C780D4B012C31
:10BAF00001D0062C08D10C79012C04D0022C02D0E4
:10BB0000072030BC70475C705B78012B03D0022BA0
:10BB100004D00520F5E730BCFFF782BB30BCFFF74F
:10BB200079BC00003028002003484179002901D069
:10BB3000012101717047000030280020BFF34F8FB2
:10BB400005480168054A01F4E06111430160BFF353
:10BB50004F8F00BFFDE700000CED00E00400FA0588
:10BB60002DE9F041204A034640F6FF76106B516BF9
:10BB700000F580550C1A04F6FF746FF30B0406EB06
:10BB800094066FF30B06C71821B1884202D100203A
:10BB9000BDE8F081904608B9C8F84870A64203D9BC
:10BBA00004F6FF70060B3603324639462846FFF787
:10BBB00083FE0028ECD1324639462846FFF762FE64
:10BBC0000028E5D135443744A64201D9002400E0DD
:10BBD000A41BD8F834100020091BC8F8301000F05E
:10BBE000C5F8002CDAD1D3E77030002038B1054910
:10BBF00001600549416001210172002070470E205B
:10BC0000704700000DBC07003FBC070030B402467F
:10BC1000112039B10B78052B05D2DFE803F00E06B1
:10BC20000C0E0E000E2030BC70470220087030BC95
:10BC3000104600F04DB81120F5E70820F3E7024662
:10BC4000112041B10B78022B04D1022A05D0032A1E
:10BC500000D1082070470E207047002003220A7090
:10BC60007047000070B50B480024D0F85C11491CE7
:10BC700003D1D0F89C01401C09D04FF4FE25284682
:10BC800000F046FA57220349284600F059FA2046A8
:10BC900070BD00007030002010B528B11C2203498F
:10BCA000FCF703FC002010BD0E2010BD9CF1070026
:10BCB00010B5064C00221821201DFEF755FB216807
:10BCC000814201D1012010BD002010BD9CF1070070
:10BCD00070B50C4D0400D5F89C0105F5CE7503D068
:10BCE000401C03D0082070BD0E2070BD002218211A
:10BCF000201DFEF739FB206007222146284629DF58
:10BD000070BD000000F00700002258210148FEF736
:10BD10002BBB00007430002070B5FFF7FBFC08B1AE
:10BD2000FDF7E6FF4FF4DC752A460E490E48FCF796
:10BD3000BCFB0D4C2068401C04D0FFF7E5FF2168D8
:10BD400081420ED029460848FCF7C8FB01206060FC
:10BD5000002000F00BF8002803D0BDE87040FDF78C
:10BD6000C7BF70BD00F007007030002070B50446FA
:10BD7000002201210C48FFF7BDFC90B9FFF7C4FF7A
:10BD80000A494FF4DC752A460860A1F5DC70FCF71F
:10BD90008CFB23462A4606490348FFF7C9FC0028C6
:10BDA00000D0032070BD000000F0070070300020BC
:10BDB000B82E002070B50848084D401BC60800206A
:10BDC000044606E005EBC40040688047002802D125
:10BDD000641CB442F6D370BDCCDD0700C4DD07009F
:10BDE00070B50848084D401BC6080020044605E011
:10BDF00055F834008047002802D1641CB442F7D3C0
:10BE000070BD0000CCDD0700C4DD070070B50F4C2D
:10BE10000025207808B1852516E00021A160616029
:10BE20002161E1604FF0E020D0F80001012610F020
:10BE3000010F03D10721002000F070F800F03CFA58
:10BE400008B9034806602670284670BD48320020B5
:10BE50001805004008B500208DF800006846FEF780
:10BE60005FF80648C168491EC160C06808B9FEF79E
:10BE700069FE9DF80000FEF777F808BD4832002003
:10BE8000F8B5174D0446A878002648B114B161688A
:10BE9000012088478DF800606846FEF741F817E0FA
:10BEA0008DF800606846FEF73BF824B10C48214647
:10BEB0001030FEF725FEE86850B94FF48270FEF7A7
:10BEC0005FFF02204107C1F8040306490120086012
:10BED000E868401CE8609DF80000FEF745F8F8BDF2
:10BEE000483200200800004010B500F011F84FF073
:10BEF00080414FF0FF30C1F80803FEF723FEFEF744
:10BF000099FD02490020087010BD00004832002051
:10BF10004FF0E0210120C1F8800170474907090E68
:10BF2000002806DA00F00F0202F1E02282F8141D68
:10BF300003E000F1E02282F8001400F01F0201216A
:10BF400091404009800000F1E020C0F88012C0F864
:10BF5000001170472DE9F0411F46154604000E46BA
:10BF600016D02068B8B1C5B160680268501E304272
:10BF700015D16A432046FDF764FE80B120683B4638
:10BF80002A46D0F810C031462046BDE8F04160474F
:10BF90000E20BDE8F0810820FBE70920F9E710201A
:10BFA000F7E720B119B101600B68114618470E2060
:10BFB00070470000044801214174007A08B1002054
:10BFC000704701207047000070340020012801D024
:10BFD000032808D10449002201284A7400D0002017
:10BFE000087400F0FBBE70477034002070B5244C1C
:10BFF0000246207A012835D002283FD1214800236B
:10C00000022A006802D0032A2CD119E0E3600179EA
:10C0100011B1012926D10BE0D0E90565711B142966
:10C0200000D31421294481614569A9420ED019E049
:10C030000169491C01614269914213D1237217E0E1
:10C04000E168491CE16008290CD9E3602372022AE7
:10C050000ED00D21FEF774FC0B480A49091D00683B
:10C06000FEF73AFE607C28B1BDE8704000F02AB9C6
:10C070000021EFE7BDE8704000F0B0BE70BD0000E9
:10C0800070340020A4280020FCDA07002DE9F843D2
:10C090001D46089F1646884604000DD066B12068EC
:10C0A00060B135B160684068B5FBF0F100FB11503C
:10C0B00030B10920BDE8F8830E20FBE70820F9E73E
:10C0C0004046FDF7B8FD90B13046FDF7B4FD70B1C4
:10C0D0002A4641462046FDF7B4FD40B1009720684E
:10C0E0002B463246C76841462046B847E2E7102053
:10C0F000E0E74FF0A04202EB80000321C0F80017F8
:10C1000070474FF0A04201218140C2F808157047E6
:10C11000094902220A60BFF36F8FBFF34F8F0A1DD8
:10C12000106006480268002AFCD000200860BFF3B7
:10C130006F8FBFF34F8F704704E5014000E401406B
:10C1400070B50E4C01232360BFF36F8FBFF34F8F89
:10C1500000230B4D08E000BF51F8236040F8236036
:10C160002E68002EFCD05B1C9342F5D3002020608B
:10C17000BFF36F8FBFF34F8F70BD000004E5014028
:10C1800000E4014020B103490968016000207047C4
:10C190000E207047A4DC070060DF704730B593B015
:10C1A0005FF03805ADF8445011A903A861DF30B144
:10C1B000052816D013B0BDE83040FDF799BD03AC9B
:10C1C0000949684600F0AAF807E000BFD0E900215D
:10C1D00020469047684600F0B8F802980028E1D061
:10C1E000F4E713B030BD0000A8DC070010B50D4C1B
:10C1F0002078A0B10120A07000F0C0FF11280CD061
:10C20000022000F0D3FF11DF002807D12070A070BA
:10C2100001F084F9032000F0C9FF002010BD0820C0
:10C2200010BD0000AC28002038B5174C207808B1AC
:10C23000082038BD0125A570002000F09FFF1128BF
:10C2400020D0002000F0B2FF104811490068009093
:10C25000684610DF0028ECD12570A07060700721BF
:10C26000162000F03FFF08B1FDF742FD0721152021
:10C2700000F038FF08B1FDF73BFD01F06BF901203C
:10C2800000F094FF002038BDAC2800203CDC070003
:10C29000ED9C07000EB50749684600F03FF805E041
:10C2A000D0E900108847684600F04FF8029800284F
:10C2B000F6D10EBD58DC0700014800787047000039
:10C2C000AC2800200548817819B1007818B1FFF733
:10C2D0008DBF08207047FFF7A7BF0000AC280020E3
:10C2E0001FB5684648DF30B1052814D004B0BDE85A
:10C2F0001040FDF7FDBC084901A800F00FF806E06A
:10C30000D0E900210098904701A800F01EF803989A
:10C310000028E6D0F4E71FBDC4DC0700016009680F
:10C320004160AFF3008010B5D0E900215368994215
:10C3300001D1002104E0D1E90034A34202D0194622
:10C34000816010BD08314160F0E7816800290BD0A1
:10C35000026892680A44826041684B689A4203D13D
:10C3600008314160FFF7DFBF704700002DE9F04161
:10C3700004461348134BC01A0C21B0FBF1F6A06918
:10C380004FF0FF3110F8022C02B92169002011E0B2
:10C3900000EB400503EB85052F68974209D14F1C40
:10C3A00002D06F688F4204D194E80F00AD68A847AF
:10C3B00003E0401CB042EBD301202060BDE8F081D7
:10C3C00018DE07000CDE070010B586B0044600201A
:10C3D0000090019002900390049005900B7B3748E9
:10C3E000072B67D2DFE803F0660429351E66490093
:10C3F0004A89062A01D0032212E042888280487BC3
:10C4000004904A7CD1F80E0003A962F31F600590E6
:10C4100001208DF80C006A460020FFF765FB0246FC
:10C4200001213DE003208DF80C006A4603A900209D
:10C43000FFF75AFB0246042132E04A89032A01D061
:10C44000032204E0B1F80D10418081800122022115
:10C4500026E004208DF80C006A4603A90020FFF7AF
:10C4600043FB0246012801D0032119E0DDE9011256
:10C47000204600F08DFD06B010BD4889022801D08D
:10C4800003220CE0487B049006208DF80C006A46DD
:10C4900003A90020FFF728FB0246012804D006214B
:10C4A000204600F0D3FDE6E79DE80E00204600F0B0
:10C4B0009BFDE0E703221946F2E700006828002010
:10C4C00010B50D4C2078002814D10C4A01210C48DD
:10C4D000FDF796FC08B1FDF70BFC0948002208386F
:10C4E00040F266618068FDF7C7FC08B1FDF700FC0B
:10C4F0000120207010BD00003028002019CF070057
:10C500004CDA070030B587B00024019402940394FC
:10C5100004948A1D8B790831022B35D15388858983
:10C52000AB4231D1127A042A2ED0062A2CD0052A09
:10C530002AD0022201238DF804208DF80A300B89BD
:10C54000ADF80C304B890C31CDE90414ADF8142052
:10C55000104DADF80E30CDF818D0018A05AA288804
:10C56000A5DF18B96846FDF747FE30B1ADF80840C1
:10C5700001A92888A8DF50B106E040F2FD10ADF80F
:10C58000080001A92888A8DF002007B030BD0120DD
:10C59000FBE700006828002030B50546C888AA8857
:10C5A00087B0904223D10020059003900490009022
:10C5B000029002208DF8000001F112000190088A1B
:10C5C000029003AA69460020FFF78EFA094C6088A2
:10C5D00000280CD0A088401E0004000CA08006D1CA
:10C5E000DDE90412284600F0D3FC6088A08007B083
:10C5F00030BD000068280020F8B50D4614460646F8
:10C60000694600F057FA00280ED0009BFF2B0AD88D
:10C61000581C834207D869780222B2EB911F02D0DE
:10C620002979814201D20020F8BD2370611C304677
:10C63000009A00F069FBF8BD114600F0D6B811462B
:10C6400000F0E3B8F8B50C4615460646694600F01A
:10C6500031FA00280CD0009A501C904207D3617820
:10C660000223B3EB911F02D02179814201D2002035
:10C67000F8BD2946304600F047FB009A0021A95436
:10C68000F8BD2DE9FF410C468E6817460546694600
:10C6900000F00CFB00280ED0A06800280BD06078BA
:10C6A0003A46C0F3011002283146684606D000F031
:10C6B000DBF80199696004B0BDE8F08100F086F80C
:10C6C000F7E77CB50D461446694600F090F900285E
:10C6D00020D02879082806D0042809D002280AD0BA
:10C6E00001280CD015E0DDE90001C4E900010AE0F1
:10C6F0000098206006E0009800B2208002E00098D8
:10C7000040B22070C117DDE9002350405940084372
:10C7100001D000207CBD01207CBD7CB50D461446B7
:10C72000694600F0A2F9002820D02879082807D00F
:10C730000021042809D002280AD001280CD014E0D6
:10C74000DDE90001C4E9000109E00098206006E08D
:10C75000009880B2208002E00098C0B22070DDE92D
:10C76000002350405940084301D000207CBD0120E7
:10C770007CBD7CB50D461446694600F076F900286C
:10C7800021D02979082908D00098C21704290BD094
:10C7900002290DD001290ED014E0DDE90002C4E920
:10C7A00000020146134609E0C3170146206005E078
:10C7B00001B2218001E041B22170CB1741405340CA
:10C7C000194301D000207CBD01207CBD70B50D4611
:10C7D000064614461146284600F083FA22462946AA
:10C7E0003046BDE8704000F03FB838B50C46042232
:10C7F000694600F089FA002806D09DF803100098D9
:10C8000061F31F602060012038BD1CB50C46082272
:10C81000694600F079FA002824D09DF801109DF8AF
:10C8200000209DF80230080E42EA012242EA03424B
:10C8300040EA13409DF803309DF8041040EA1320AD
:10C8400008439DF8051042EA036240EA01209DF882
:10C85000061040EA01409DF8071040EA0160C4E973
:10C86000002001201CBD00002DE9F04F04469DB0C2
:10C8700000200090064601904FF0FF3A0AA800F011
:10C8800051F94FF0010BE94682E012AB05AA06A967
:10C89000204600F0C9F850B10AA8059900F053F9F4
:10C8A00060B10B98407810F0300F53D060E09DF8E5
:10C8B0004800002870D11DB0BDE8F08F0598B04247
:10C8C00042D30B9D0AAE0B98407800F00F00082869
:10C8D00012D0304600F04EF90B98A842F3D15646DC
:10C8E0000599B14230D3D4F8088009919DF8181009
:10C8F00008910E990D6820E00B980678F0E72968FA
:10C900000F682FB1DDE9083229462046B84711E00B
:10C9100011948968DDE90872097891420CD12946A1
:10C9200017A8FEF7F8F885F80CB017AA3946119841
:10C93000FDF777FD0028BED0AD6815B1A16841456F
:10C94000DDD0A168414523D19DF81810204600F0A4
:10C9500017FA1BE00C9840280AD200F01F010BFACE
:10C9600001F00C994A0959F82230034349F8223062
:10C97000E5682DB10AAB9DF8182020460599A84717
:10C980000AAA9DF818102046FDF74BFD002892D00A
:10C99000A06800287FF479AFDDE90B0445780AA888
:10C9A00000F0E8F80028F7D115F0300F03D10B980C
:10C9B000007800B1641CC4B10020494605E000BF06
:10C9C00051F82020521C0ED1401CB0EB541FF7D35D
:10C9D000600959F8201004F01F00C0F120022AFA63
:10C9E00002F0814201D0002065E7012063E71CB519
:10C9F0000C46694600F039F8002814D0DDE9000241
:10CA0000C10709D051084FEA30006FEA00026FEA0F
:10CA10000100C4E9002004E051084FEA3000C4E9F5
:10CA200000014FF001001CBDF8B50746002018704A
:10CA300008700E4610601C4615466946384600F0E0
:10CA400039F801004FF0010009D0009959B1C80828
:10CA50002860009800F0070030700120F8BDB96828
:10CA600009B10020F8BD2070FBE72DE9F84300264E
:10CA7000884681463446354604E0402E02D30020E5
:10CA8000BDE8F8836946484600F06AF90028F7D007
:10CA90009DF80070324607F07F00C10FFBF7F6FCEF
:10CAA00029430443F61D0D463806E6D4C8E9004183
:10CAB0000120E5E7F8B50E460746694600F050F953
:10CAC00000280AD09DF80040200616D5072504F05E
:10CAD0007F0403E0202D01D30020F8BD69463846CD
:10CAE00000F03EF90028F8D09DF8001001F07F001A
:10CAF000A8400443ED1D0806ECD401203460F8BDC5
:10CB00005968064A8968914206D1D0E90110044A61
:10CB1000401E491CC2E9001070470000F0D8070011
:10CB200040280020C26000230160C0E901138B7817
:10CB30001A44026191F903301A44426108780028CE
:10CB400000D00120704770B545680E460446606805
:10CB50000178B14206D1407800F00F00082801D0DA
:10CB6000012070BD204600F005F86068A842EED1B3
:10CB7000002070BD30B541680A785AB101F10C034C
:10CB800043600A7B42B14C780A79C4F30115032D46
:10CB900007D00BE0002030BDC2680168FFF7C2FF7C
:10CBA000F8E75D78C5F30115032D07D00225B5EB35
:10CBB000141F09D14C7914FB02F209E08D78046945
:10CBC0000022641B046103E0B5EB941F00D1042232
:10CBD000497811F0300F02D18168491C81609C783E
:10CBE000016921441144016193F903201144416119
:10CBF000012030BD30B54168002487B0497801F08C
:10CC00000F02082A11D08A091ED00222B2EB911F0E
:10CC100009D10269C1F301110229146001D003296D
:10CC200001D14069047007B030BD0069056808E0B3
:10CC30002C7329466846FDF76EFF6846FFF7DAFF5A
:10CC4000AD68002DF4D1EEE7C1F30111012912D036
:10CC50000229E6D00329E4D04268517801F00F019F
:10CC600007290BD0916881B11279006907B0BDE83E
:10CC70003040FBF71ABC41690C70EDE70169906820
:10CC800007B0BDE8304000F02CB81179006907B05A
:10CC9000BDE83040FBF722BC10B5034B002408C0B0
:10CCA00080E8160010BD000079A2070038B50D46D7
:10CCB00004466946FFF7FEFE00280BD0D4E90002C7
:10CCC000D4E90213C5E90002C5E9021300988142C4
:10CCD00001D2002038BDA860A168081AA060012018
:10CCE00038BD00B50A4687B001466846FFF71AFF0F
:10CCF000002807D06846FFF77DFF6846FFF73AFF38
:10CD00000028F7D107B000BD7FB514460546A9B984
:10CD1000124A2868904208D110E01022694628463D
:10CD2000FFF7F2FF002807D0103C102CF5D8224660
:10CD300069462846FFF7E8FF04B070BDA868A04226
:10CD400001D20020F8E72B682246284698470028A1
:10CD5000F2D0A868001BA8600120EDE779A20700C7
:10CD600010B504468068002809D0236801222046B7
:10CD70009847002803D0A068401EA060012010BD85
:10CD800038B5002439B1012912D0022912D0052961
:10CD90001DD0002038BD0546012269462846FFF710
:10CDA000B3FF90B19DF800000006F5D4012038BD16
:10CDB00008220DE005466946FFF77CFE28B10021F8
:10CDC0002846009AFFF7A0FF38BD204638BD042250
:10CDD000BDE838400021FFF797BF00002DE9F04182
:10CDE000204C0025204E207A012730B91F48311DE4
:10CDF0000068FDF77CFF306038B102202072316896
:10CE0000087928B101281CD114E06560BDE8F081E3
:10CE1000D1E90503C01A142800D31420B7EB900FF2
:10CE200001D2820800E001220869C9681844194447
:10CE300029DF03E0D1E90301084428DF38B11128D4
:10CE40000ED003213068FDF77BFD2572DDE7207CE5
:10CE50000028DBD1BDE8F04100210220FFF7C6B871
:10CE60002772D3E770340020A4280020FCDA0700E2
:10CE700038B5084C0121201D6A46FBF79DFA009049
:10CE8000002806D1607C002803D1BDE83840FFF7B8
:10CE9000A5BF38BD7034002010B510461A46FBF708
:10CEA00004FB002010BD10B510461A46FBF7FDFA32
:10CEB000002010BD2DE9F0411E681C4615460746AE
:10CEC00021B1012918D0052923D119E000202060C3
:10CED000401C2060B0421CD8012229463846FFF78A
:10CEE00013FF002806D015F8010B000601D52068B5
:10CEF000EEE70120BDE8F08108200246186002E05C
:10CF000004200246186029463846BDE8F041FFF784
:10CF1000FBBE0020EEE700000A4810B500790028AB
:10CF20000ED0FEF747FFBFF34F8F07480168074A4F
:10CF300001F4E06111430160BFF34F8F00BFFDE7D3
:10CF400010BD0000302800200CED00E00400FA05C0
:10CF500010B5FEF71FF9002814D00B4A00210B482A
:10CF6000FCF74EFF08B1FCF7C3FE084800224FF45F
:10CF7000A0210068FCF780FF002803D0BDE8104026
:10CF8000FCF7B6BE10BD00003DBB0700C4DA0700C9
:10CF90002DE9F041124D0646904628880A46A0F534
:10CFA0007F41FF3919D0287AC00716D00D4C602078
:10CFB0000121207003206070A170E11C104600F078
:10CFC000FBFBC71CE119404600F0F6FBC219B18912
:10CFD0002888BDE8F04100F015B90820BDE8F081CF
:10CFE00068280020182D00202DE9F047154D064631
:10CFF000904628880A46A0F57F419946FF391ED001
:10D00000287AC0071BD0104C602006212070617068
:10D010000120A070E11C104600F0CEFBC71CE119F6
:10D02000404600F0C9FB0744E119484600F0C4FB44
:10D03000C219B1892888BDE8F04700F0E3B808209C
:10D04000BDE8F08768280020182D00202DE9F04168
:10D05000114D07462888A0F57F43FF3B0BD0287A67
:10D06000C00708D00D4C6020032620706170A270AC
:10D070000B2A03D009E00820BDE8F081FDF788FC09
:10D08000E07004260020FDF78BFCB9893246288821
:10D09000BDE8F04100F0B6B868280020182D002047
:10D0A000084670470846704770B5012670044FF077
:10D0B000E0210025C1F88001084C4010C4F8480365
:10D0C000C4F8080366602F20FDF7D0FFA660044C6B
:10D0D0002F20A560FDF7CAFFA57070BD00100140AC
:10D0E0008C28002070B50D460446FCF787FD70B112
:10D0F0002846FCF795FD68B16807000E002C0CDA95
:10D1000004F00F0101F1E02181F8140D09E042F271
:10D11000010070BD42F2020070BD04F1E02484F809
:10D120000004002070BD000038B50021012558B171
:10D1300001280ED003280BD107210020FEF7EEFEB8
:10D14000BDE83840FEF786BE4FF0E020C0F88051C1
:10D1500038BD8DF800106846FCF7E2FE064C2078DA
:10D1600008B9FEF753FEE068401CE060A5709DF82A
:10D170000000FCF7F9FE38BD483200203EB50446F9
:10D1800009496846FFF7CAF808E000BFD0E9002166
:10D190002046904730B16846FFF7D7F8029800283C
:10D1A000F4D13EBD11203EBD40DC07003EB5044633
:10D1B00008496846FFF7B2F807E000BFD0E9002150
:10D1C000204690476846FFF7C0F802980028F5D13E
:10D1D0003EBD00004CDC0700084907480860010715
:10D1E0004FF08070C1F80C050548002240F6CD4193
:10D1F0008068FCF741BE00003546526E00060140D3
:10D2000078DA070007B584B000220092ADF800106C
:10D2100001218DF8021006A90291034903910192A0
:10D220006946A6DF07B000BD182D002070B5164670
:10D230000D46040007D035B1206C8022002138282B
:10D24000225403D307E00E2070BD2154401C38281F
:10D25000FBD30BE02154401C4028FBD32146084659
:10D2600000F096F838212046FBF738F9216CD4E914
:10D2700012304A0FC900383459185041C4E904101B
:10D28000227CE2710A0A42EA0062A2710A0C42EAB6
:10D2900000426271020242EA116020716069E0702E
:10D2A000010AA170010C6170000E04F838092146D2
:10D2B000084600F06DF84FF00002EEB1E06ED100CC
:10D2C000C840A854A36ECB40A8180371636ECB402E
:10D2D0000372236ECB400373E36DCB400374A36DE5
:10D2E000CB400375636DCB400376236DCB40521C5E
:10D2F0000377042AE2D31FE018235042216D03EB89
:10D30000C000C140A954666DC640A9180E71A66D33
:10D31000C6400E72E66DC6400E73266EC6400E7491
:10D32000666EC6400E75A66EC6400E76E66EC640A8
:10D33000521C0E77042AE0D3002070BDA8B1002152
:10D340000164C0E912110A4901650A4941650A49A7
:10D3500081650A49C1650A4901660A4941660A4967
:10D3600081660A49C166002070470E2070470000A0
:10D3700067E6096A85AE67BB72F36E3C3AF54FA566
:10D380007F520E518C68059BABD9831F19CDE05B92
:10D390002DE9F04FC8B0002213466F46CC181B1D74
:10D3A0002568E4782DBA25F0FF05254347F822507B
:10D3B000521C102AF2D31BE007EB820151F8083C03
:10D3C0004FEA734484EAF34484EA932451F83C3CE2
:10D3D0004FEAF31585EAB34585EAD303234451F8B0
:10D3E0001C4C51F8401C2144194447F82210521C8F
:10D3F000402AE1D3036D4793416D4691846D459476
:10D40000C26D44929246026E4392456E4295A94681
:10D41000856E4195C66E4096B34600264FEAB21718
:10D4200087EAF22787EA726C02EA090725EA02080E
:10D4300087EA0807BC44204F57F8268008EB0B0703
:10D44000BC445DF82670AB460CEB070E4FEAB30701
:10D4500087EA733787EAB35C81EA04074D4601EA3D
:10D46000040891461F400AEB0E02A24687EA08070D
:10D470000C46BC441946761C0EEB0C03402ECDD353
:10D48000479E33440365469B1944416545992144B1
:10D49000816544995144C16543991144016642999B
:10D4A0004944416641992944816640995944C1667D
:10D4B00048B0BDE8F08F00002CDB07002DE9F041FB
:10D4C00016460F46040004D006B317B10025A8463F
:10D4D0001AE00E20BDE8F081216C785D6054206C6C
:10D4E000401C206440280ED121460846FFF750FF1B
:10D4F000D4E912014FF40072801841F10001C4F820
:10D500004080C4E912016D1CB542E5D30020E1E77B
:10D51000002801D1FCF7BEBE7047000010B51620F0
:10D52000FCF76CFB48B10A4882684FF4800152B1A5
:10D53000016821F48001016010BDBDE8104042F295
:10D540000100FCF7D5BB4FF0E020C0F8801110BD02
:10D550006833002010B51620FCF750FB80B10F484F
:10D5600090F800044009FCF75BFB60B10C4882684E
:10D570004FF480016AB1016841F48001016010BD7F
:10D5800042F2010001E042F20200BDE81040FCF767
:10D59000AFBB4FF0E020C0F8001110BD16E000E076
:10D5A000683300200C4910B50A4808600B4C002273
:10D5B0004FF480316068FCF75FFC002240F6CD41FB
:10D5C000A068FCF759FC4FF0A0414FF08070C1F803
:10D5D0000C0510BD3546526E0006014078DA070092
:10D5E0002DE9F84F1D4C00256846D4E901A6FDF74A
:10D5F00021F9002738B30023009A61681CE0D1F8B4
:10D6000000C00846944503D9ACEB02020A6015E05D
:10D61000A2EB0C0263440760D0F80CC0C1698146DC
:10D62000BCF1000F08D006EB030828F07F48C0E9E2
:10D63000018CC9F81C5005460029E0D128466160DC
:10D64000FDF794FA03E02846FDF790FA10B1504632
:10D65000FCF734FEE770BDE8F88F00008C2800204E
:10D660000D4B10B5596831B102680C68A24204D85C
:10D67000A21A0A60C161586010BD0B4603E00B4658
:10D68000C969121B21B10C689442F8D3A41A0C602A
:10D690000260C161D86110BD8C2800202DE9F041E5
:10D6A000144E77683D462C4603E0844204D025465C
:10D6B000E469002CF9D11BE0D4B1A5420BD1F86983
:10D6C000706040B90C49012088600021B160F070A1
:10D6D0002F20FDF7CBFC2168E069E86110B10268FA
:10D6E000114401607068874202D00120BDE8F081DA
:10D6F0000020FBE78C280020001001407CB5064686
:10D7000000240D468DF800406846FCF709FC01A88E
:10D7100000F074F870B10570094946609DF8040086
:10D7200048709DF80000FCF71FFC1420FCF75AF825
:10D7300020467CBD04249DF80000FCF715FCF7E7AB
:10D740005C3200202DE9F041194D6C68002C2CD082
:10D75000184800270068A968B846401A20F07F469C
:10D760002068B0420CD82146361A0744E469087C88
:10D7700020B181F81080886949698847002CEFD171
:10D7800029786878814206D1401CC0B268700228AE
:10D7900001D185F80180064869780C3040F8217085
:10D7A000BDE8F0411420FCF71DB8BDE8F081000091
:10D7B0008C280020041501400870020A4A70020CEF
:10D7C0008A70000EC87004207047000010B502482F
:10D7D000FDF7A3FA002010BDA028002010B51421E9
:10D7E0000448FAF77BFE04480068FDF74FFA002072
:10D7F00010BD000070340020FCDA07000A494A78A6
:10D800008B78521CD2B2934200D100220B78934203
:10D8100001D1002070470270487800EB400001EB16
:10D82000C000001D704700005C32002000207047DF
:10D83000002070472DE9F84380461C4617460E46E7
:10D840000C48089DFDF770FA10B11120BDE8F8836F
:10D85000A20839463046FEF773FC0648FDF75DFA2C
:10D8600023463246012140460095FDF74DF8002041
:10D87000ECE70000A02800202DE9F84F114D884664
:10D8800081461E4617466946DDF828A02868FDF740
:10D8900018FA040013D01C21FAF720FE0020207192
:10D8A000C4F80090C4E90486C4E902A76946286860
:10D8B000FDF728FAFFF7DCFA0020BDE8F88F042016
:10D8C000FBE70000FCDA0700000000000101000097
:10D8D000010000000000000002050000210000001F
:10D8E0000000000000000000000000000000000038
:10D8F000011104FC0400000000000000021104FCFF
:10D900000400000000000000032104FC04100000DB
:10D9100000000000041101FF0100000000000000F1
:10D92000051102FE0400000000000000061104FCC6
:10D930000400000000000000071104FC04000000C7
:10D9400000000000081701FF22000000CCD80700EB
:10D95000091001FF01000000C8D807000000000006
:10D9600000000000000000000101000004000000B1
:10D9700000000000000000000000000000000000A7
:10D98000011101FF0100000000000000021702FE6B
:10D9900094000000F0D80700031704FC0400000006
:10D9A00068D907000000000000000000000000002F
:10D9B00001070000A000000080D90700020100005C
:10D9C000010000000000000003050000410000000D
:10D9D0000000000000000000000000000000000047
:10D9E000011704FCA000000080D90700021704FC06
:10D9F000E4000000B0D907000000000000000000B3
:10DA00000000000033CE8A374C153ACC3AFE14D0D1
:10DA1000D29AC57F3FC1291AA02F71F3386126EC35
:10DA20009A83DE820903516CC7E50DD71382536ECA
:10DA3000FD48D99719ACD5A64D517C90491ABAEE3C
:10DA4000C7B5F5FA0500040500000000642C0020AD
:10DA500002000000000000000000000000000000C4
:10DA6000000028000000000050EADA308883B89FE8
:10DA7000604F15F30000C98E482D0020682D00204E
:10DA8000882D0020010000000000000000000000C0
:10DA90000000000002000000000000000000000084
:10DAA0000000000003000000000000000000000073
:10DAB0000000000004000000000000000000000062
:10DAC000000000002832002000000000700000006C
:10DAD00000100000040000000100000091AA0700EF
:10DAE000CDD7070099CE070035D8070075A80700E5
:10DAF000A1D007002DD80700D5AA07008434002044
:10DB00000010000004000000010000009DAA0700B2
:10DB1000DDD70700A7CE070079D80700BDA807000A
:10DB2000A5D0070031D80700E5AA0700982F8A4240
:10DB300091443771CFFBC0B5A5DBB5E95BC256395F
:10DB4000F111F159A4823F92D55E1CAB98AA07D877
:10DB5000015B8312BE853124C37D0C55745DBE729A
:10DB6000FEB1DE80A706DC9B74F19BC1C1699BE41A
:10DB70008647BEEFC69DC10FCCA10C246F2CE92DAA
:10DB8000AA84744ADCA9B05CDA88F97652513E98CE
:10DB90006DC631A8C82703B0C77F59BFF30BE0C6D5
:10DBA0004791A7D55163CA0667292914850AB72763
:10DBB00038211B2EFC6D2C4D130D385354730A6500
:10DBC000BB0A6A762EC9C281852C7292A1E8BFA2D7
:10DBD0004B661AA8708B4BC2A3516CC719E892D13F
:10DBE000240699D685350EF470A06A1016C1A419C2
:10DBF000086C371E4C774827B5BCB034B30C1C39C1
:10DC00004AAAD84E4FCA9C5BF36F2E68EE828F747F
:10DC10006F63A5781478C8840802C78CFAFFBE9099
:10DC2000EB6C50A4F7A3F9BEF27871C6D4DD0700FF
:10DC3000DCDD07000000000000000000010000071C
:10DC40002CDC07003CDC07000800000064DC070057
:10DC500074DC07000800000074DC070084DC0700A7
:10DC600008000000FCDD07000CDE070000000000DB
:10DC700000000000ECDD0700FCDD070000000000F4
:10DC80000000000000000000000000000000000094
:10DC900000000000CCDD0700D4DD0700000000001C
:10DCA000000000003028002084DC0700A4DC07000E
:10DCB00008000000DCDD0700ECDD070000000000CC
:10DCC00000000000B4DC0700C4DC0700080000000E
:10DCD00073C707001BC70700C3C6070039C6070084
:10DCE0003FC60700F9C5070045C6070083C6070001
:10DCF0000000000008200001FFFFFFFFFFFFFFFF03
:10DD0000FFFFFFFF00000000000000000000000017
:10DD100001000000FFFFFFFF512563FCC2CAB9F3F9
:10DD2000849E17A7ADFAE6BCFFFFFFFFFFFFFFFFD2
:10DD300000000000FFFFFFFF96C298D84539A1F40C
:10DD4000A033EB2D817D0377F240A463E5E6BCF8B8
:10DD500047422CE1F2D1176BF551BF376840B6CB83
:10DD6000CE5E316B5733CE2B169E0F7C4AEBE78E7F
:10DD70009B7F1AFEE242E34F4B60D2273E3CCE3BF4
:10DD8000F6B053CCB0061D65BC86987655BDEBB396
:10DD9000E7933AAAD835C65ACD8607005F970700A1
:10DDA0007595070018DE0700302800209800000055
:10DDB000DC9B0700B0DE0700C8280020D02B000045
:10DDC000EC9B070045A0070005A00700A5A00700E1
:10DDD00000000000B5BF07000000000011D50700DB
:10DDE00000000000EDBF0700000000009DC107001B
:10DDF00000000000E1C207000000000029D1070078
:10DE000000000000CDBF070000000000000000007F
:10DE100003000000EDBB070000010000000000004F
:10DE200000000000000000000000000000000000F2
:10DE300004DA070040000000842C002040000000AD
:10DE4000C42C002020000000E42C00202000000052
:10DE5000FFFF0000000000000000000000000000C4
:10DE600000000000000000000000000000000000B2
:10DE700000000000000000000000000000000000A2
:10DE80000000000000000000000000000000000092
:10DE900000000000000000000090D003000000001F
:10DEA00000000000F5A507000010000000000800B9
:020000041000EA
:041014000080070051
:020000041000EA
:0410180000E00700ED
:04000005000782016D
:00000001FF
